:020000040000FA
:0A0000007B2800000000000009004A
:06000A00A31423102630B0
:1000100084000530A4002315A001051E0D28A101B0
:10002000051E1928A10A000068302102031C1028AF
:100030000134A10123182428051A2C28AE302102EE
:1000400003180234A10A1C28051E2C28AE302102F8
:1000500003180234A10A24280130A3062230210209
:10006000031C033468302102031C3928A31C3D28DB
:1000700004340230A306A3181928231D4E28231C7C
:100080004628201EA00AA5201928093423110C3067
:100090002002031C0A340A30A0001928A003031907
:1000A0005B2801302006031D58282318192807341F
:1000B000230CA20D19282318083422088000840A72
:1000C000A40B4B280034263084000430A400030124
:1000D0000007840AA40B68282A02031D7028003434
:1000E0000C349A302602031D7A28E9302702031DBA
:1000F0007A2800340D348501860110306500003007
:10010000660064008730620007309F008101AA20EA
:10011000A5200520FF39031D92286320FF39031D08
:1001200092287120A200A208031D882829080739F7
:100130000F3A8500A90DA90D3F30A904C03028044D
:100140002905FF3A8600B0208828811F0800810118
:10015000A50B0800A3130F30A50085018601080038
:08016000A3170F30A5000800F1
:04016800003400342B
:02400E00B13FC0
:00000001FF
